:0A0000007CC0FECFFDCF15C2FBCF80
:10000A00FACFF9CFF8CFF7CFF6CFF5CFF4CFF3CFBA
:10001A00F2CF39C250C250C2EECFEDCFECCFEBCF08
:10002A00EACFE9CFE8CFE7CFE6CF3F065B4F666D71
:10003A007D077F6F777C395E79717350583E7758A8
:10004A003E0000300000735C1C3058743E045400BB
:10005A0077744F7773713E3807070305070406075D
:10006A0000051003001017001414141414141414A7
:10007A003C3C60047E049C04B004C404D804F60426
:10008A001405320550057805030609030406080A13
:10009A00050A38CF07388766380686774F007766AD
:1000AA0000777D00777F0077063F737D0073065BDC
:1000BA0000001C0C480DAC0DDE0D100E560EA60EDF
:1000CA00000F5A0FBE0F0410200001002D4E414EA2
:1000DA0000494E46000002000200BA0016008001E4
:1000EA00BC000100FD01D20001000602D40000009C
:1000FA00F894EE27EFBBE5BFF8E1A895A4B7A77F70
:10010A00A4BFF0936000E09360008DE0A2E0BB27FB
:10011A00ED938A95E9F780E092E0A0E0B1E0ED93F3
:10012A000197E9F7E0EEF0E085919591009761F08B
:10013A00A591B59105901590BF01F00105900D921A
:10014A000197E1F7FB01F0CFE0E0EEBBEFEFEDBF87
:10015A00E2E0EEBFC0E8D1E0E1C1AA93E881F0E0B5
:10016A00EE59FF4FE491EF70E06CE0937C00E09170
:10017A007A00E064E0937A00E0917A00E071E1F3BA
:10018A00E0917A00E061E0937A00E0917800F091E2
:10019A0079004CC01A9310E01A3068F40CD5E9566D
:1001AA00FE4F0DD508D510D5A0E0A08304D50FD5F4
:1001BA0006D51F5FF1CFE2E04E2EF1980BD57724DA
:1001CA00E0E0E093E801E093E9010AD5E0E0E0939A
:1001DA00F601E4E60CD5E89422F821F80BD50DD502
:1001EA00E89426F8F49AF39AF29A27F8552409D54E
:1001FA00E0E0E093FE01E093FF01E0930002A8E152
:10020A00B0E0DBD6E03011F0E93C08F004C0A8E128
:10021A00B0E0D3D601C0E2E3E093050203C1AA939A
:10022A00E881EC1511F4E0E801C0E0E021960895B8
:10023A00BA93AA931A9310E0EAD4AF3FEFEFBE073E
:10024A0031F4E6E8E7D4E0E8E8D4EAD449C0EFEFCD
:10025A00CE2EDDD4A73EE3E0BE0748F0E4D47AD63A
:10026A001E2FE1D43AD6E983FA83C394F2CFA12FA1
:10027A00E5E0F7D5CCD4F0E0DAD4E983FA83C7D441
:10028A00E4E6F0E02AD6309739F0D4D4EF93A0E030
:10029A00C6DFAF91EA2B01C0E0E0BCD4B8D4E4E6F3
:1002AA00F0E058D6E983FA83E091E401E03021F4E2
:1002BA00BAD413D6309749F0B6D40FD6BBD4EF933D
:1002CA00A1E0ADDFAF91EA2B01C0E0E0A9D4ABD445
:1002DA0041D6B0D4EF93A2E0A2DFAF91EA2B9DD42E
:1002EA00188123960895BA93AA931A93A7D4A5E0DE
:1002FA00B0E0A083B183A7D40080118088D44ED601
:10030A000E161F0610F49AD45AD411E01B30B0F41A
:10031A009AD400801180E12F7AD49AD4AE0FBF1FED
:10032A003DD60E161F0640F089D4BF01AAE01A9FD7
:10033A00F001DB01F0E090D41F5FE8CFEB81E03001
:10034A0099F47CD4FF93EF9360817181A091B201FB
:10035A00B091B301E8ECF0E0C0D5DF01FB01EA1B84
:10036A00FB0BAF91BF9178D41881259608951A9303
:10037A00E0E350D4ECE554D4E1E74FD470D472D41E
:10038A001E2FE8EEF3E072D4ACEEB1E074D476D46A
:10039A00309781F1A0E01E99A1E0E0E0F299E1E056
:1003AA00EA1751F0E8E8F3E161D41E9902C0F29825
:1003BA0001C0F29AF29B1F5FA0E01F99A1E0E0E062
:1003CA00F399E1E0EA1751F0E8E8F3E14FD41F9915
:1003DA0002C0F39801C0F39AF39B1150A12FBB27D7
:1003EA0027DFA1E0B0E01AD51C9903C01C9BFECF01
:1003FA0001C0CACF37D4E11759F0ACE1B0E0E12F20
:10040A00E7D5EDE607D4ECE10BD4EEE506D427D424
:10041A0009C01A93EDE6FED3E9E702D4E8E7FDD373
:10042A001ED4A5DF199108952DD41E9B0AC01F9BC7
:10043A0008C0A091F901B091FA01A033E5E7BE071F
:10044A0009F427D4A0E01D99A1E0E0E030FCE1E046
:10045A00EA1729F01ED4E8941D99689430F820D43C
:10046A0023C0E0E0E4BDE2E0E5BDE091FD01E7BDC7
:10047A00E0916E00E260E0936E00E0916E00E16050
:10048A00E0936E000895FED326FC07C0A9EFB1E001
:10049A000DD4E133A5E7FA0738F0E0E3F5E7E09396
:1004AA00F901F093FA0107D4E991EFBFF991E991C3
:1004BA00B991A991189518950A921A92AA93EA9352
:1004CA00FA93EFB7EA93F7D3FCD3F0E0EC51FE4F7F
:1004DA00E081EBB9E5B1EE60E5B915B0F2D3EF5FB3
:1004EA00A1E0B7D4E095E121E5B9F09B03C0ECD3D4
:1004FA00E07809F401C05F9AA091E701AF5FA09389
:10050A00E701A33018F0E0E0E093E701E991EFBFDB
:10051A00F991E991A99119900990189520E831E08B
:10052A0039DEEFE0E4B9EEEFE5B9E7E0E7B9E0E09C
:10053A00E8B9EBB9EFEFEAB9E7E8E0937A00E0EC63
:10054A00E0937C00E8E3E0937E0041982898429883
:10055A004098E5E0E3BFF894E0E0E0936900EDBB82
:10056A00E1E0E0936800E0EFE0936B00E1E0EBBBD1
:10057A00789477DF1F9902C01E9B01C00CC010E05F
:10058A00A12FE0E2A4D3A7D334F4A12FA0D3EFEF95
:10059A001FD51F5FF5CF1E9B3CDFA1D3E0E0E093A0
:1005AA000102E0930202E0930302E0930402A7E04F
:1005BA00B0E03EDEECE92ED3A8EEB3E02FD4F099FA
:1005CA0007C0ABEFB1E072D3E739A0E0FA0708F44D
:1005DA003BC0E0E0EBB929982A982B98EAB9EBB925
:1005EA008895E89431F81C9904C0ABEFB1E043D385
:1005FA0045D31CEFEBE6F0E0E4911E177CF41030D3
:10060A0019F4EEE9F1E0DBD2A1E0A7DDA0919E01A9
:10061A00B0919F010CD369D31F5FECCFE0919E018B
:10062A00F0919F0167D369D360D374D3A0919901E4
:10063A00B0919A01FDDDE3E7EDD2EFEFEAB91E9B37
:10064A0002C01F9901C0FBCFF09B46C069D3AA30F4
:10065A0080F069D368F0AAEEB1E028D3A091EA014C
:10066A00B091EB01509718F0B5D2E0E0C0D201C0CA
:10067A00B1D2E091F701E03021F4289AE1E0B7D253
:10068A005DD34ED3A13049F4A091F801A53010F4FE
:10069A0059D303C053D3E2E0AAD242D3A23049F4D9
:1006AA0042D320F0F19A289AE4E601C0E3E0E0930D
:1006BA00F70136D3A33021F441D32898E4E097D246
:1006CA002FD3A43049F4A091F801A83210F43AD3F8
:1006DA0003C034D3E0E08BD21DD37724E8E07E1642
:1006EA0008F03FC235D3E03009F439C2F59B04C0A3
:1006FA00A2EEB1E0DBD201C031D3E42DF0E0EE5836
:10070A00FF4FE491A091E201B091E301E4D258F0E5
:10071A00F598E8E0E41539F427D3E03021F4F69AA5
:10072A00E1E0E093F601F69B04C0A0EFB1E0BED28F
:10073A0001C01DD3A091F001B091F101A036E0E013
:10074A00BE0788F0E0E9F0E031D40ED3E150F0E0E2
:10075A00EE56FF4FE491FF2766277727B4D30DD3D0
:10076A00F79AF69804D3F79B04C0A2EFB1E09ED2A1
:10077A0001C008D3A091F201B091F301A036E0E0E4
:10078A00BE0730F110E01B300CF5E12FA8ECB1E008
:10079A005FD24DD2FF93EF93E12FACE7B0E058D28E
:1007AA0046D204D488279927E091EE01F091EF010F
:1007BA00A1D28ED3DF01CB01E0E9F0E0F3D39AD2E4
:1007CA00C4D3AF91BF9148D21F5FDDCFF798F09A9B
:1007DA0010E0BED2EC5FA12F7AD27DD20CF0BFC15D
:1007EA00A72DBBDCE093E001F093E101D1D2DF0158
:1007FA00EC91EF5FEC93CCD2A081A53050F0CDD232
:10080A00E956FE4F0F01DF01C9D3CCD210D2D00175
:10081A0023D2BED2A0819CD2EC5FAE17F8F0BDD233
:10082A00DF01D5D1FF93EF93A956BE4FB7D362D25A
:10083A0064D2AF91BF9110D2ABD2A0E0A083ADD267
:10084A00E956FE4FBCD1AED2AF3FE3E0BE0731F46A
:10085A00A4D2BDD1AFEFBFEFA083B1831E9B05C069
:10086A00B39409F4BA9466240DC0639409F46A94A3
:10087A00BB24F29B07C066241F9902C0689421F822
:10088A00689424F81F9B05C0A39409F4AA94992498
:10089A000DC0939409F49A94AA24F39B07C099244F
:1008AA001E9902C0689422F8689423F81C9B05C01C
:1008BA00D39409F4DA94882409C0839409F48A94B5
:1008CA00DD24F49B03C08824689425F81E9902C08D
:1008DA00F29801C0F29A1F9902C0F39801C0F39AE4
:1008EA001C9902C0F49801C0F49A21FC02C022FEAD
:1008FA0018C0E89421F822F8E0E58CD1EDE690D111
:10090A00E8E78BD11E9B02C01F9901C0FBCFF0986C
:10091A0041982898F698F798E89420F8E0D13ADCBC
:10092A003CCE1D9902C0F09B01C01AC09BD1A09178
:10093A00A801B091A901CFD150F4AEEDB1E0B6D182
:10094A00309721F4AEEDB1E096D198D101C059D1DA
:10095A002ED228F0E0E0E093FB01E093FC0101C015
:10096A0050D1A091DE01B091DF01A33CEAE3BE07BA
:10097A0010F01DD208F403C0419A43D101C0419836
:10098A0025FE1BC020FE07C0E0E6F0E0E093F4017C
:10099A00F093F5012FD1F79B07C0E0E6F0E0E09372
:1009AA00F201F093F30126D1F69B07C0E0E6F0E0EE
:1009BA00E093F001F093F1011DD125FE15C0539487
:1009CA00E2E0E51508F45524A52DE0E04FD2E03029
:1009DA0011F4429801C0429AA52DE1E047D2E030D5
:1009EA0011F4409801C0409A24FC06C067FE03C077
:1009FA006BD1EF7109F033C053D1F79B0AC0C2D152
:100A0A00DED1A138EEE3BE0718F4DED110D1B5D19C
:100A1A0026C020FE09C0DDD1A538E3E0BE0718F4E0
:100A2A00E2D1359623D11BC0F69B0CC0A091F601EA
:100A3A00AA3018F499D1EF5F01C0E1E0E093F60122
:100A4A0096D10DC0E0E0E41510F44A9402C0E8E043
:100A5A004E2EE4E0E41509F44A94C2D0BBD023FC3C
:100A6A0006C097FE03C030D1EF7109F034C018D127
:100A7A00F79B0EC087D1A3D1A93EE3E0BE0738F0A9
:100A8A00A3D1AE1BBF0BA093EE01B093EF0123C01D
:100A9A0020FE07C09ED1159718F0A5D13597E6D04C
:100AAA001AC0F69B0CC0A091F601A23018F05CD1D6
:100ABA00E15001C0EAE0E093F60159D10CC0E8E048
:100ACA004E1610F4439401C04424E4E0E41509F4FA
:100ADA00439486D07FD08ED090D0F19B08C0419AA3
:100AEA003DD1F098E4E683D0F598E7E04E2EF59BE9
:100AFA0009C07ED1E42DA3E0EA9FF001EC5BFF4F31
:100B0A007ED122C0F69B0AC073D12ED1E150A3E058
:100B1A00EA9FF001E456FF4F72D116C0F79B02C05C
:100B2A004ED111C020FE05C0A091EC01B091ED019B
:100B3A000AC031FE09C0E42DA5E0EA9FF00147D0C2
:100B4A00DF012CD2DF0174DBBFD0EF5FE09300023C
:100B5A00E03019F4AEEFB1E0A9D01F5F3ACE73943A
:100B6A00BDCD689431F827FC03C0DAD0AB3038F039
:100B7A00E2E0EA93E8E0EA93A8ECB1E0B4DBE091C2
:100B8A00A801F091A90141D153D1E0930102F09358
:100B9A0002026093030270930402AEE1B0E009D24C
:100BAA003196E254F54D31D1ABD1E093BC01F093CB
:100BBA00BD0105CDFFCFA5E01A9FF0010895A0E081
:100BCA00B0E0A083B1830895EA56FE4F0895E75630
:100BDA00FE4F0895E0E0E093EA01E093EB01089507
:100BEA00F59AE0E0E093E201E093E3010895E093EF
:100BFA00F7010895E89425F80895E89424F823F86D
:100C0A000895E0E0E093DE01E093DF010895A98111
:100C1A00BA810895E093E4010895E093E601089506
:100C2A00E093E5010895F3DFEAE0F0E00895EA0FC2
:100C3A00FB1F0895EC5CFF4FE4910895EB81A5E05A
:100C4A00EA9FF001C4CFEC81A5E0EA9FF001BFCF93
:100C5A00F0E0EE0FFF1F0895ED93FC930895ACEDBD
:100C6A00B5E0DCC0ACE1B0E0A8D10895E093EC01B6
:100C7A00F093ED010895ED91FD9108953197FE935A
:100C8A00EE930895AA93BA93EA93FA93EFB7EA9385
:100C9A000895EFEFFFEFE093FB01F093FC01089555
:100CAA00E0E0E093F901E093FA010895E4DF319678
:100CBA00FE93EE930895299A2A9A2B9AE0E0EBB9CB
:100CCA000895E091E7010895E09100020895B0E0E7
:100CDA00A7FDBFEF0895F0E0AE17BF070895E0E063
:100CEA00E093EC01E093ED010895E0939E01F09307
:100CFA009F010895662777270895ACE4B4E080E061
:100D0A0090E0C1D0DF01CB01E0E0F4E060E070E008
:100D1A00F7D00895E1E0EA93E0E0EA93D901E3CA63
:100D2A00A091F7010895E091A301F091A401A09187
:100D3A00EE01B091EF01EA17FB070895E0E0E093B6
:100D4A00F8010895E091F801EF5FE093F801089542
:100D5A00E72DF0E0E659FF4FE4910895E0E0E093D3
:100D6A00E201E093E3010895E091F6010895E0E0DD
:100D7A00E093F001E093F1010895E093EE01F0931E
:100D8A00EF010895E0E0E093F201E093F3010895A2
:100D9A00E72DA5E0EA9FF00117CFE72DA5E0EA9F2E
:100DAA00F0010895A091E001B091E1010895A091A8
:100DBA00A301B091A401A93EE3E0BE070895A09162
:100DCA00EE01B091EF010895E0910502F8DFF0E03D
:100DDA000895E0E0E093F401E093F501A091EC01BD
:100DEA00B091ED010895E091EC01F091ED010895C3
:100DFA0068DFF0E0CF01EC51FE4FBF010895E80F24
:100E0A00F91FE491DB01EC930895A0910102B091DE
:100E1A00020280910302909104026CCF109639F07D
:100E2A0080E491E00197F1F7A8951197C9F7089521
:100E3A00EA0FFB1F681F791F0895F195E195F040AD
:100E4A000895F09560957095E195FF4F6F4F7F4F2C
:100E5A000895EE230E2EEA2F19F0EE0F0A94E9F701
:100E6A000895AE17E1E008F4EE270895EA17E1E0E5
:100E7A0008F0EE270895FA9FF02DEB9FF00DEA9FF8
:100E8A00E02DF10D08957A9F702D6B9F700DF89FDC
:100E9A00700DE99F700D6A9F602D710DFB9F600DAB
:100EAA00711DE89F600D711D8827FA9FF02D610D55
:100EBA00781FEB9FF00D611D781FEA9FE02DF10D61
:100ECA00681F781F089549D0D6DF0EF4B6DF08955B
:100EDA0052D0D9DF0EF4B5DF08950024112490E131
:100EEA00AA0FBB1F001C111C0E1A1F0A18F40E0EA3
:100EFA001F1E01C0A1609A9599F7FD01D0010895BE
:100F0A003F934F935F93002411244427552730E2DF
:100F1A00AA0FBB1F881F991F001C111C441F551FB5
:100F2A000E1A1F0A460B570B28F40E0E1F1E461FD9
:100F3A00571F01C0A1603A9559F7FD01BC01D001C4
:100F4A00CA015F914F913F91089515D0D9DF0EF4F0
:100F5A0078DF0895C2DFFD010895E894F7FF02C023
:100F6A006CDF6894B7FF06C0A095B095119600F89B
:100F7A00039400FA0895E89477FF02C062DF689448
:100F8A0097FF0BC00024A095B09580959095119677
:100F9A00801D901D00F8039400FA0895ED91FC91CC
:100FAA00119708950590F491E02D0895A591B491B3
:100FBA000895119602D0FE2F1197F999FECFFF934B
:100FCA00FFB7F894A1BDF89AE0B5FFBFFF91089565
:100FDA00F99B02C0A895FCCF9FB7F894A1BDF89AD7
:100FEA0080B5E81719F0E0BDFA9AF99A9FBF0895FB
:00000001FF
